:1000000010C02AC029C028C027C026C025C024C0CF
:1000100023C0FBCC21C05DCD1FC01EC01DC01CC0B5
:100020001BC011241FBECFE5D2E0DEBFCDBF10E064
:10003000A0E6B0E0E0E7FBE102C005900D92A83633
:10004000B107D9F711E0A8E6B0E001C01D92A937C9
:10005000B107E1F7C7DC8ACDD3CF282FAA98AB9898
:100060003A9A00003A9883B390E034E096958795E9
:100070003A95E1F7817090E027FF02C0AA9A01C08B
:10008000AA9867FF02C0AB9A01C0AB983A9A0000E9
:100090003A98973019F0880F9C9981609F5F98304B
:1000A00019F0220F660FE8CFAA98AB983A9A000091
:1000B0003A9800003A9A00003A980895AF9A0000E2
:1000C0000000AF980895AD9800000000AD9A089523
:1000D000AC9AA99A00000000A998AC980895982FAE
:1000E00080916C00833021F4892F6CE4B6DF089591
:1000F000AA9A8FEF8ABB9BBBAF9A00000000AF9813
:10010000AA981ABA1BBA0895982F80916C00833070
:1001100021F4892F6CE0A1DF08958FEF8ABB9BBB90
:10012000AF9A00000000AF981ABA1BBA0895982F32
:1001300080916C00833021F4892F6CE18EDF08956B
:10014000AC9A8FEF8ABB9BBBAF9A00000000AF98C0
:10015000AC981ABA1BBA0895982F80916C0083301E
:1001600021F4892F6CE279DF0895AB9A8FEF8ABB77
:100170009BBBAF9A00000000AF98AB981ABA1BBAAD
:100180000895982F80916C00833021F4892F6CE3BF
:1001900064DF0895AC9AAB9A8FEF8ABB9BBBAF9A92
:1001A00000000000AF98AC98AB981ABA1BBA08953B
:1001B0000F931F9380916C00833049F580E068E6CF
:1001C0004CDF009168001091690080E06CE645DF2B
:1001D000F801EC58FF4F80830F5F1F4F10936900A9
:1001E0000093680080E068E738DF009168001091B4
:1001F000690080E06CE731DFF801EC58FF4F808345
:100200000F5F1F4F109369000093680022C0AE98E3
:100210000000809168009091690029B3FC01EC58BE
:10022000FF4F208301969093690080936800AC9AF9
:100230000000809168009091690029B3FC01EC589E
:10024000FF4F208301969093690080936800AE9AD7
:10025000AC981F910F9108950F931F9380916C009C
:100260008330A9F480E068E6F8DE00916800109120
:10027000690080E06CE6F1DEF801EC58FF4F808306
:100280000F5F1F4F109369000093680011C0AE9874
:100290000000809168009091690029B3FC01EC583E
:1002A000FF4F208301969093690080936800AE9A77
:1002B0001F910F9108950F931F9380916C008330CD
:1002C000A9F480E06AE6C9DE009168001091690037
:1002D00080E06EE6C2DEF801EC58FF4F80830F5FCE
:1002E0001F4F10936900009368001FC080916C003D
:1002F000813011F4A89A01C0AA9AAE9800008091AA
:1003000068009091690029B3FC01EC58FF4F2083ED
:1003100001969093690080936800AE9A80916C007A
:10032000813011F4A89801C0AA981F910F910895E7
:100330000F931F9380916C008330A9F480E068E7ED
:100340008CDE009168001091690080E06CE785DE2A
:10035000F801EC58FF4F80830F5F1F4F1093690027
:100360000093680013C0AC9AAE98000080916800BA
:100370009091690029B3FC01EC58FF4F208301964E
:100380009093690080936800AE9AAC981F910F918A
:1003900008950F931F9380916C008330A9F480E03F
:1003A0006AE75BDE009168001091690080E06EE70B
:1003B00054DEF801EC58FF4F80830F5F1F4F1093FE
:1003C00069000093680021C0AC9A80916C00813074
:1003D00011F4A89A01C0AA9AAE9800008091680012
:1003E0009091690029B3FC01EC58FF4F20830196DE
:1003F0009093690080936800AE9AAC9880916C00ED
:10040000813011F4A89801C0AA981F910F91089506
:10041000399892B782B7891B8532E0F3389A3298BF
:100420003A9814BA15BA1ABA1BBA089586B18360FD
:1004300086B9389A399832983A9814BA15BA1ABACD
:100440001BBA81B38C6381BB82B3837C82BB87B3CD
:10045000886B87BBC69AC39AC49A10BC83E089B9DB
:1004600088ED8AB9E4E7F0E0119281E0E937F80716
:10047000D9F7109269001092680080916A0081603B
:1004800080936A0083E083BF7894929A089590BD28
:1004900089B988ED8AB90895882319F0813021F44B
:1004A00002C0C39A0895C398089592B782B7891B72
:1004B0008532E0F3C49A80E0EFDF1DB81EB80895DE
:1004C000873008F086E0E82FF0E0E05AFF4F908197
:1004D000892F80658DB996FF02C0709A0895709833
:1004E00008951DB81EB808958FB9779BFECF089563
:1004F0001FB8779BFECF8FB10895EF92FF920F93B5
:100500001F9300E05CEAE52E43E5F42EC498C798FB
:1005100081E0C2DF90E022B782B7821B8532E0F330
:100520009F5F9134C1F7802FCBDFEFB8779BFECF71
:10053000FFB8779BFECF1FB8779BFECF8FB1833577
:1005400011F010E002C0102F1F5F1FB8779BFECF85
:10055000C49A80E0A1DF1DB81EB8112319F40F5F03
:100560000730A1F6812F1F910F91FF90EF90089512
:100570003091770020E080917800280F311DC9016B
:10058000089598E49093740096E590937500809395
:10059000760070937700609378000895789481E0F6
:1005A00090E090936900809368005D9BFECF8091FE
:1005B00074008CB908959091770080E020917800C4
:1005C000820F911D25E030E0309369002093680090
:1005D000892BA9F480916A0082FF11C080916A0082
:1005E0008F7B80936A0080916A008B7F80936A0082
:1005F00080916C00843011F40BDF01C056DF88E479
:100600008093740086E58093750088ED8093760072
:100610001092770010927800C1DF08951F93182F71
:1006200080936B0092989398949A80916A00806866
:1006300080936A0080916A008F7B80936A0080912A
:100640006A0083FF0AC080916A00877F80936A00F6
:1006500080916C00843009F0DBDE80916A0082FFBB
:100660000AC080916A008B7F80936A0080916C0041
:10067000843009F0CDDE88E48093740086E58093B1
:1006800075008FEE809376001092770081E0809362
:1006900078001093790082DF1F91089580916D009A
:1006A000882349F1C498C79881E0F6DE90E022B72C
:1006B00082B7821B8532E0F39F5F9134C1F780914E
:1006C0006D008150FDDE8CEA8FB9779BFECF83E50C
:1006D0008FB9779BFECF1FB8779BFECF8FB11FB826
:1006E000779BFECF833511F480E00895DEDE82E053
:1006F00095DF8FEF089587E091DF8FEF0895CEDFCC
:100700008F3FC9F08CEA8FB9779BFECF80E88FB915
:10071000779BFECF1FB8779BFECF1FB8779BFECF8E
:1007200090E022B782B7821B8532E0F39F5F983258
:10073000C1F7BBDE80E008950F931F93AFDF8F3FBB
:1007400009F45FC09091770080E020917800AC01BF
:10075000420F511D415050405695479560E070E062
:100760000CEA10EEB4EAA8EA30EA45C080916800CD
:1007700090916900FC01EC58FF4F20810196909305
:100780006900809368008091680090916900FC0185
:10079000EC58FF4FE08101969093690080936800C8
:1007A0000FB9779BFECF213021F43FB9779BFECF65
:1007B00011C0223021F4AFB9779BFECF0BC023309C
:1007C00021F4BFB9779BFECF05C0243019F41FB9BF
:1007D000779BFECF1FB8779BFECFEFB9779BFECFFD
:1007E00090E022B782B7821B8532E0F39F5F9F3093
:1007F000C1F76F5F7F4F6417750708F4B7CF55DEF9
:1008000080E01F910F9108951F9348DF8F3F09F4F7
:1008100075C060E070E018E5B0E5A8E05FC0E09169
:100820006800F0916900EC58FF4F8181813089F4B4
:10083000BFB9779BFECF1FB8779BFECF1FB8779BC2
:10084000FECF20916800309169001FB8779BFECFE2
:1008500038C0823089F41FB9779BFECFAFB9779B40
:10086000FECF1FB8779BFECF2091680030916900C2
:100870001FB8779BFECF25C0833089F4BFB9779B23
:10088000FECFAFB9779BFECF1FB8779BFECF2091ED
:100890006800309169001FB8779BFECF12C084308A
:1008A000D9F41FB9779BFECF1FB8779BFECF1FB837
:1008B000779BFECF20916800309169001FB8779B2D
:1008C000FECF8FB1F901EC58FF4F80832F5F3F4F70
:1008D00030936900209368006F5F7F4F50917700DD
:1008E00040E0809178009A01280F311DC9010197DD
:1008F0006817790708F493CFD8DD80E01F91089539
:10090000CDDE8F3F29F188E38FB9779BFECF1FB8EB
:10091000779BFECFE0916800F0916900EC58FF4FA3
:1009200081818FB9779BFECF20916800309169005B
:100930001FB8779BFECF8FB1F901EC58FF4F808332
:100940002F5F3F4F3093690020936800AEDD80E059
:100950000895A4DE8F3F11F190E040E34FB9779BFB
:10096000FECF1FB8779BFECF9FB9779BFECF20911C
:100970006800309169001FB8779BFECF8FB1F901F5
:10098000EC58FF4F80832F5F3F4F309369002093D7
:1009900068009F5F933011F788DD80E008958091B3
:1009A0006A008F7780936A0088E48093740086E5FC
:1009B0008093750080ED80937600109277001092FE
:1009C0007800ECDD0895F89480916A00806480934B
:1009D0006A009298939A0895F6DF80916A008F7B5F
:1009E00080936A0081E08093790010927A0088E415
:1009F0008093740086E5809375008BED809376007C
:100A00001092770082E080937800C8DD0895DBDFE4
:100A100080916A008F7B80936A0081E080937900E7
:100A200092E090937A0088E48093740086E5809346
:100A300075008AED8093760010927700909378008D
:100A4000ADDD0895C0DF8091790080936D008091C5
:100A50006A008F7B80936A0088E48093740086E547
:100A60008093750089ED809376001092770081E085
:100A70008093780093DD0895A6DF3FDD80936D00BD
:100A800080916D008093790080916A008F7B8093C4
:100A90006A0088E48093740086E58093750089ED90
:100AA000809376001092770081E08093780076DD65
:100AB0000895FF920F931F9380916A0086FD12C0E4
:100AC00082DFECDD8F3F09F4E7C080916A00886027
:100AD00080936A0088E48093740086E580937500B3
:100AE00085EDD3C09091770080E020917800DC0103
:100AF000A20FB11D40E050E070ECF72E00E418E4C6
:100B00007CE460E06BC08091720090917300209152
:100B10006F0030E0289FA001299F500D389F500D95
:100B20001124460F511D80916E008130A1F50FB93F
:100B3000779BFECF1FB8779BFECF342F4FB9779BA3
:100B4000FECF8091680090916900FC01EC58FF4F46
:100B50002081019690936900809368002FB9779B5C
:100B6000FECF1FB9779BFECF1FB8779BFECF3FB953
:100B7000779BFECF8091680090916900FC01EC5852
:100B8000FF4F2081019690936900809368002FB9F0
:100B9000779BFECF22C0FFB8779BFECF5FB9779BD4
:100BA000FECF4FB9779BFECF80916800909169008E
:100BB000FC01EC58FF4F20810196909369008093CF
:100BC00068002FB9779BFECF90E022B782B7821BD7
:100BD0008532E0F39F5F9E31C1F76F5F80916F00B8
:100BE000681708F490CF242F952F80916E008130E4
:100BF000A9F47FB9779BFECF9FB9779BFECF2FB922
:100C0000779BFECF1FB8779BFECF90E022B782B7CD
:100C1000821B8532E0F39F5F9F30C1F780917200A5
:100C200090917300019690937300809372002091CD
:100C300072003091730080917000909171002817BC
:100C4000390798F032DC80916A008F7B80936A00CC
:100C500080916A00877F80936A0088E480937400A3
:100C600086E58093750087ED10C0809168009091B3
:100C7000690005978A179B0708F443CF88E480939F
:100C8000740086E58093750086ED8093760010925F
:100C900077001092780080E01F910F91FF900895E7
:100CA0001F9380916A0086FD0AC08DDEF7DC8F3FBE
:100CB00009F4AAC080916A00846080936A0060E0B1
:100CC00010EAB0E2A8E25EC08091720090917300D9
:100CD00020916F0030E0289FA001299F500D389F80
:100CE000500D1124460F511D80916E00813071F519
:100CF000BFB9779BFECF752F5FB9779BFECF942F3F
:100D00004FB9779BFECF20916800309169001FB8E2
:100D1000779BFECF8FB1F901EC58FF4F80832F5F97
:100D20003F4F3093690020936800AFB9779BFECFA7
:100D30007FB9779BFECF9FB9779BFECF209168004C
:100D4000309169001FB8779BFECF10C01FB9779B09
:100D5000FECF5FB9779BFECF4FB9779BFECF209137
:100D60006800309169001FB8779BFECF8FB1F90101
:100D7000EC58FF4F80832F5F3F4F309369002093E3
:100D800068006F5F80916F00681708F49DCF8091B5
:100D9000720090917300019690937300809372009B
:100DA00020917200309173008091700090917100D9
:100DB0002817390760F080916A008F7B80936A0062
:100DC00080916A008B7F80936A006FDB19C09091DD
:100DD0006F0080916E00823029F0292F30E0220FC1
:100DE000331F04C080916F00282F30E0809168008D
:100DF000909169000597820F931F8150914010F0E8
:100E000080E003C060E0BECF8FEF1F910895EF92A6
:100E1000FF920F931F93D7DD41DC8F3F11F41FEF3B
:100E20009EC010E0A0EAEA2EF0E2FF2E08E2A5E064
:100E3000B0E060E074C080917200909173002091E6
:100E40006F0030E0289FA001299F500D389F500D62
:100E50001124460F511D80916E00813009F043C06E
:100E6000B0936900A0936800FFB8779BFECF752F01
:100E70005FB9779BFECF942F4FB9779BFECF209120
:100E80006800309169001FB8779BFECF8FB1F901E0
:100E9000EC58FF4F80832F5F3F4F309369002093C2
:100EA00068000FB9779BFECF7FB9779BFECF9FB9C4
:100EB000779BFECF20916800309169001FB8779B27
:100EC000FECF8FB1F901EC58FF4F80832F5F3F4F6A
:100ED0003093690020936800809179008F3F91F4EE
:100EE00080917A000DC0EFB8779BFECF5FB9779BFA
:100EF000FECF4FB9779BFECF1FB8779BFECF8FB148
:100F00008F3F59F0809170009091710001979093FC
:100F100073008093720011E007C06F5F10E0809152
:100F20006F00681708F487CF80917200909173006A
:100F3000019690937300809372002091720030911B
:100F4000730080917000909171002817390708F4A0
:100F500070CF80916A008F7B80936A00A6DA812F20
:100F60001F910F91FF90EF90089585E090E090938E
:100F7000690080936800E0916800F0916900EC5886
:100F8000FF4F808180936C001EDD08958091790071
:100F900080936C0080917A0080936E0080917B003A
:100FA00080936F0090917C0080E020917D00820F03
:100FB000911D9093710080937000109273001092B5
:100FC000720008951F93182F80916C00833051F4A4
:100FD00080E090E001969C990FC020E48030920759
:100FE000C9F70FC080E090E001962A9905C020E47F
:100FF00080309207C9F705C08050904411F080E01E
:1010000004C006DA812F0ADB8FEF1F9108958FEF5E
:1010100084BB15BA80916C00833079F4329A3A9887
:10102000389892B782B7891B8532E0F3399A81E309
:101030008A95F1F7A498AC9810C0389880E0AF9AE0
:1010400000000000AF988F5F8A30C9F7399A82E0BC
:10105000B9DF8F3F41F0AE9AAD9A92B782B7891B44
:101060008532E0F380E008951F93CF93DF93809162
:101070006A0086FD6EC0A7DCCADF8F3F09F46BC033
:1010800080916A00846080936A0063C080917200DE
:101090009091730020916F0030E0289FE001299F1C
:1010A000D00D389FD00D1124C10FD11D80916E003D
:1010B000813011F482E001C083E011D88C2F24D854
:1010C0008D2F35D880916E00813011F471D801C018
:1010D000C3D81F5F80916F001817C0F28091720013
:1010E0009091730001969093730080937200209109
:1010F00072003091730080917000909171002817F8
:10110000390760F080916A008F7B80936A0080913C
:101110006A008B7F80936A007BD919C090916F0021
:1011200080916E00823029F0292F30E0220F331F8A
:1011300004C080916F00282F30E08091680090916A
:1011400069000597820F931F8150914010F080E055
:1011500003C010E0BFCF8FEFDF91CF911F910895B3
:101160009091770080E020917800AC01420F511DF2
:1011700085E090E0909369008093680041155105E7
:1011800099F480916A0082FD16C088E4809374000F
:1011900086E58093750088ED809376001092770045
:1011A00010927800FBD908954530510521F48091C3
:1011B0006A0082FFEBDE80916C00843021F470DDE8
:1011C0008F3F21F4089550DF8F3F99F080916800A0
:1011D00090916900059728E42093740026E52093F8
:1011E000750024ED2093760090937700809378002B
:1011F000D5D90895EF92FF920F931F93CF93DF936A
:10120000E2DB05DF8F3F11F41FEF65C010E000E067
:1012100085E0E82EF12C3EC0809172009091730021
:1012200020916F0030E0289FE001299FD00D389F6A
:10123000D00D1124C00FD11DF0926900E09268001A
:1012400080916E00813011F482E001C083E047D7C5
:101250008C2F5AD78D2F6BD780916E00813041F43F
:10126000A7D7809179008F3F41F480917A0003C025
:10127000F3D7809179008F3F59F080917000909161
:1012800071000197909373008093720011E007C082
:101290000F5F10E080916F00081708F4BDCF8091B8
:1012A0007200909173000196909373008093720086
:1012B00020917200309173008091700090917100C4
:1012C0002817390710F400E0E5CF80916A008F7B82
:1012D00080936A009DD8812FDF91CF911F910F914C
:1012E000FF90EF9008959091770080E02091780032
:1012F000820F911D25E030E0309369002093680053
:10130000059781F543DE80916C00843011F47FDD18
:1013100001C070DF282F85E090E0909369008093F2
:1013200068008091680090916900FC01EC58FF4FC3
:1013300020830196909369008093680080916800F3
:1013400090916900059728E42093740026E5209386
:1013500075002CED209376009093770080937800B1
:101360001DD9089581E05AD90895EF92FF921F93F5
:10137000CF93DF934CDE8F3F69F1EE24FF241BC037
:10138000E0916800F0916900EC58FF4F118184E012
:10139000A6D6113011F460D70BC0123011F4F9D772
:1013A00007C0133011F487D703C0143009F4C0D735
:1013B0000894E11CF11CD0917700C0E08091780086
:1013C0009E01280F311DC9010197E816F906C0F2E8
:1013D0001FD880E0DF91CF911F91FF90EF9008958B
:1013E000C4DD80916C00843021F40EDA8F3F21F44B
:1013F0000895BBDF8F3FC1F080916A008F7B80939F
:101400006A008091680090916900059728E4209314
:10141000740026E52093750023ED209376009093C9
:10142000770080937800BAD80895F1DD8F3F69F096
:1014300088E055D6E0916800F0916900EC58FF4FC4
:10144000818162D675D7E4D780E008958EDD8091E2
:101450006C00843021F454DA8F3F21F40895E5DFE5
:101460008F3FA1F080916A008F7B80936A0088E4AF
:101470008093740086E58093750082ED80937600FA
:101480001092770081E08093780088D808951F93A8
:10149000BEDD8F3F59F010E088E021D6812F34D691
:1014A000DBD61F5F1330C1F7B3D780E01F910895DB
:1014B0005CDD80916C00843021F44BDA8F3F21F4A5
:1014C0000895E5DF8F3FA1F080916A008F7B8093C4
:1014D0006A0088E48093740086E58093750081ED4E
:1014E000809376001092770083E08093780056D83E
:1014F0000895FF920F931F93CF93DF9380916A001B
:1015000086FF03C0C0E0D0E0D8C05DDA80DD8F3F49
:1015100009F4DDC080916E00813011F480E101C0DA
:1015200081E1DDD580916A00886080936A0088E45B
:101530008093740086E58093750085EDA6C0809148
:1015400072009091730020916F0030E0289FE001BD
:10155000299FD00D389FD00D1124CF0DD11D8C2F78
:10156000D3D580916E00813041F520916800309193
:101570006900F901EC58FF4F80812F5F3F4F309396
:10158000690020936800E8D52091680030916900D7
:10159000F901EC58FF4F80812F5F3F4F3093690076
:1015A00020936800EED580916C00833009F580E0CF
:1015B0006DE753D580E06CE71AC08D2FB8D5209128
:1015C000680030916900F901EC58FF4F80812F5F6E
:1015D0003F4F3093690020936800BED580916C0026
:1015E000833031F480E06DE638D580E06CE635D5A7
:1015F00080916C00813009F46BD5F39480916F0079
:10160000F81608F49CCF80916E00813011F48D2F74
:101610008ED580916C00833039F480E064E61DD56E
:1016200080E06CE61AD504C0AD9800000000AD9AC9
:1016300085E0C8DC8F3F09F44AC080917200909128
:101640007300019690937300809372002091720052
:1016500030917300809170009091710028173907C4
:10166000E0F080E03CD5D4D680916A008F7B8093F7
:101670006A0080916A00877F80936A0088E4809383
:10168000740086E58093750087ED80937600109254
:1016900077001092780080E01BC0809168009091E4
:1016A000690005971091770000E020917800A8016B
:1016B000420F511D8417950710F4FF249FCF88E433
:1016C0008093740086E58093750086EDDECF8FEF02
:1016D000DF91CF911F910F91FF9008959091770026
:1016E00080E020917800820F911D25E030E030935A
:1016F000690020936800059721F480916A0083FFB8
:1017000045DC80916C00843021F4D3D98F3F21F4E3
:101710000895EFDE8F3F09F041D7089578DC8F3FC1
:10172000D1F080E8DCD480916C00833039F480E023
:1017300064E693D480E06CE690D404C0AD980000D9
:101740000000AD9A86E03EDC8F3F29F080E0C7D4F0
:101750005FD680E008958FEF089507DC80916C00DC
:10176000843021F4CCD78F3F21F40895D7DF8F3F09
:1017700099F080916A008F7B80936A0088E480935F
:10178000740086E58093750080ED8093760010925A
:1017900077001092780002D70895EF92FF920F938E
:1017A0001F93CF93DF9333DC8F3F09F494C0EE2473
:1017B000FF247EC08091680090916900FC01EC5884
:1017C000FF4F10810196909369008093680080918B
:1017D000680090916900FC01EC58FF4F0081019670
:1017E00090936900809368001430A9F480E277D464
:1017F000802FB2D480916C00833039F480E064E6AD
:101800002CD480E06CE629D404C0AD980000000020
:10181000AD9A83E047C080E462D4802F9DD411301C
:1018200079F480916C00833031F480E064E615D463
:1018300080E06CE610C0AD9800000000AD9A31C0A9
:10184000123091F480916C00833039F480E064E7C9
:1018500004D480E06CE701D424C0AC9AAD980000B9
:101860000000AD9AAC981DC01330D9F480916C0083
:10187000833031F480E066E6F0D380E06EE6EBCFB3
:1018800080916C00813039F4A89AAD980000000076
:10189000AD9AA89806C0AA9AAD9800000000AD9A2B
:1018A000AA9884E08FDB8F3FB1F00894E11CF11C13
:1018B000D0917700C0E0809178009E01280F311D03
:1018C000C901019796958795E816F90608F472CF35
:1018D0009FD580E001C08FEFDF91CF911F910F91D5
:1018E000FF90EF90089541DB80916800909169002E
:1018F0000196909369008093680080916C00843019
:1019000021F41AD78F3F21F4089547DF8F3F99F0D4
:1019100080916A008F7B80936A0088E480937400D2
:1019200086E58093750080ED8093760010927700B5
:101930001092780033D608959091760080916A00D5
:101940008D7F80936A0080916A0087FF06C09F3C6C
:1019500009F43FC080916B0043C0923381F193330F
:1019600080F4903221F1913228F49031E1F09131FC
:10197000B1F51BC09033F9F09133F8F4913279F559
:1019800018C0913C51F1923C38F4913BE1F0903C0D
:1019900011F1903B21F515C0933CC9F0933CA8F0A0
:1019A0009F3CE9F416C084DD089550DD089518DDEC
:1019B000089599DF0895D4DB0895FDD508958EDE4E
:1019C0000895CBDE08958FDC089556D808953AD84F
:1019D0000895E5D708951BD80895FED7089581E0AE
:1019E0001DD6089523D580916A0081FFFCCFA4DF26
:1019F000FACF382F90E006C022B782B7821B85321B
:101A0000E0F39F5F9317C0F308951F920F920FB6F4
:101A10000F9211242F933F934F938F939F93EF93A4
:101A2000FF9380916A0080FD02C08CB146C0959AF8
:101A300080916800909169002CB1FC01EC58FF4F37
:101A400020830196909369008093680080916800DC
:101A500090916900029769F480917400883421F4B0
:101A600080917500863549F11092690010926800E6
:101A700023C080916800909169000597F0F08091F3
:101A80006800909169003091770020E040917800E3
:101A9000240F311D05972817390779F41092690032
:101AA0001092680080916A008E7F80936A00809116
:101AB0006A00826080936A009598FF91EF919F91F0
:101AC0008F914F913F912F910F900FBE0F901F90CC
:101AD00018951F920F920FB60F9211242F933F93D8
:101AE0004F938F939F93EF93FF93959A8091680004
:101AF000909169003091770020E040917800240FA8
:101B0000311D2B5F3F4F8217930778F48091680057
:101B100090916900FC01EC58FF4F20812CB901968F
:101B2000909369008093680015C01092690010922C
:101B30006800959880916A0086FD07C080916A00D0
:101B400087FD03C094989398929A80916A0081606F
:101B500080936A00FF91EF919F918F914F913F91F8
:101B60002F910F900FBE0F901F901895F894FFCFF4
:081B7000400041014243030063
:00000001FF
